:100000001AC027C026C047C124C023C022C021C0B7
:1000100020C01FC0000102030405060708090A0BDF
:100020000C0E12171C2229313A45505D6B7B8DA0B6
:10003000B5CBE4FF400211241FBECFE9CDBF20E0C5
:10004000A0E6B0E001C01D92AA36B207E1F74FD199
:10005000B8C1D6CF42E050E060E070E087E690E0C3
:1000600084C142E050E060E070E087E690E08CC13F
:1000700042E050E064E370E087E690E06DC1F8DFB5
:10008000F0CFE8DF809167008F3F29F4809168000E
:100090008F3F09F4F4CF08958FB5806B8FBD08951D
:1000A0008FB58F778FBD8FB58F7D8FBD8FB58F7ECD
:1000B0008FBD08958FB583608FBD83B7836083BF85
:1000C000EBDF8FEF86BF89BD89B7826089BF089556
:1000D00083E487B985E886B9089548E080E090E038
:1000E000369A3699FECF24B135B1820F931F415015
:1000F000B9F723E0969587952A95E1F790936100EB
:1001000080936000089540916000509161002091BB
:100110006700309168004217530758F486B790E0A3
:10012000841B950B820F931F8F3F910578F08FEF03
:100130000DC0421B530B86B790E08417950710F44F
:1001400016BE05C086B790E0841B950B86BF86B7A8
:10015000869586958695EFE1E81BF0E0EC5EFF4F13
:10016000E491E095E9BD0895FC018081B2991AC03F
:10017000813041F018F08230F1F40EC081E08083CC
:1001800086E007C080916200811115C082E0808303
:100190008AEE809362000FC08091620081110BC0D3
:1001A00082E00895823039F48091620010828823C1
:1001B00011F081E0089580E008958091630081113D
:1001C0000AC084E690E0D0DF823039F569DF81E053
:1001D00080936300089584E690E0C6DF8130E9F4FF
:1001E0007CDF8091600090916100893A924030F00C
:1001F00088EA92E0909361008093600080916000B3
:10020000909161008F31910520F090936800809368
:10021000670027DF41DF109263000895809160003E
:10022000909161008E31910568F480916500811193
:1002300004C088E780936500C498809165008C3085
:10024000C1F414C0893A924068F080916500811130
:1002500004C088E180936500C4988091650088306F
:1002600041F404C080916300811102C0C49A01C0AE
:10027000C49880916300882369F08091690081119E
:1002800004C088E280936900C19880916900803140
:1002900009F4C19A08951F920F920FB60F9211247C
:1002A0008F93809166008F5F8093660080916600D7
:1002B0008230B9F480916200882319F081508093D4
:1002C000620080916500882319F081508093650059
:1002D00080916900882319F0815080936900109201
:1002E00066008F910F900FBE0F901F90189583E1BD
:1002F00087BB85E088BB2FEF8DEE92E021508040D8
:100300009040E1F700C00000B2990BC0B8DEC19A7E
:100310002FEF81EF9BE2215080409040E1F700C039
:100320000000AFDEC7DE2FEF8DEE92E0215080405F
:100330009040E1F700C00000CBDE2FEF8DEE92E0A1
:10034000215080409040E1F700C00000789435DFF4
:10035000C4DED9DE63DFFBCFFB01DC0102C0059008
:100360000D9241505040D8F70895A82F862FE82FBE
:10037000E199FECF1FBA05C0EEBBE09AE3950DB23E
:100380000D924150C8F70895A82FA40F415030F0A6
:10039000862F840F2E9104D04150E0F70895262F28
:1003A000E199FECF1FBA8EBBE09A81500DB20216C2
:1003B00039F01CBA2DBB0FB6F894E29AE19A0FBE41
:0603C0000895F894FFCF40
:00000001FF
